:1000000012C019C018C017C016C015C014C013C044
:1000100012C011C010C00FC00EC00DC00CC00BC06C
:100020000AC009C008C011241FBECFE5D4E0DEBF5E
:10003000CDBF8BD22EC3E4CFA998AB988823A9F06B
:10004000AA9AAB9A90E02AE109C0AA98AB9A822FAB
:100050008A95F1F79F5F983031F0660FAB9867FF94
:10006000F4CFAA9AF3CFA99A0895AA98EACF0F934A
:100070001F93182F062F80E06BE2DEDF81E0612FF7
:10008000DBDF81E0612FD8DF80E06AE2D5DF81E04D
:10009000602FD2DF81E0602FCFDF1F910F91089595
:1000A0000F931F938A01E3DF80E06CE2C5DFA9981C
:1000B000B80175956795759567957595679575956B
:1000C000679581E0B9DF02951295107F1027007FB8
:1000D000102781E0602FB0DFA99A80E060E0ACDFFC
:1000E0001F910F9108952F923F924F925F926F92BE
:1000F0007F928F929F92AF92BF92CF92DF92EF92B8
:10010000FF920F931F93CF93DF93A82EB62E242E2A
:10011000322E480130E0261B3109842F90E08A19E5
:10012000910937FD68C071E0472E512C97FD5CC0E6
:1001300061E0662E712C6901CC0CDD1C7C01EE0C9B
:10014000FF1C8A2D6B2DA401ABDFCE14DF047CF5E0
:100150002A14D1F0C70195958795E601C81BD90BE4
:10016000062D162D1A0D02C0CC0DDD1DD7FD03C0C6
:10017000B40CCE19DF09812F6B2DA40191DF100F74
:10018000812F801B281681F7DF91CF911F910F914E
:10019000FF90EF90DF90CF90BF90AF909F908F90A7
:1001A0007F906F905F904F903F902F9008953B14F9
:1001B00059F3C60195958795E701C81BD90B042D06
:1001C000142D1B0D02C0CE0DDF1DD7FD03C0A60CE4
:1001D000CC19DD098A2D612FA40162DF100F812F58
:1001E000801B381681F7D0CF909581959F4F66245C
:1001F0006A94762CA0CF309521953F4F44244A94A1
:10020000542C94CF9F92AF92BF92CF92DF92EF92F5
:10021000FF920F931F93CF93DF93D82EA62EC42E59
:10022000B22E0130F1F02A2D87015DDF8D2D6B2D6F
:100230004C2D2B2D58DF8D2D6A2D4D2D2B2D53DF61
:100240008C2D6A2D4C2D2B2D4EDFDF91CF911F91E0
:100250000F91FF90EF90DF90CF90BF90AF909F9065
:100260000895942E841708F475C00C2DCD1408F44D
:100270006BC0DB2CAB1408F461C01B2DBA1408F45E
:100280005BC080E06BE2D8DE81E0692DD5DE81E0E5
:10029000602FD2DE80E06AE2CFDE81E06D2DCCDE21
:1002A00081E0612FC9DE80E06CE2C6DE212F30E004
:1002B0002F5F3F4F2D193109802F90E0019689194A
:1002C0009109289FA001299F500D389F500D11249E
:1002D00057FD46C06A01D594C794D7FC29C0C70111
:1002E00095958795959587959595879595958795F6
:1002F000082F8F2D992787FD9A95182F1F70C701FA
:1003000082959295907F9827807F9827182BC0E040
:10031000D0E0A99881E0602F8FDE81E0612F8CDE34
:1003200081E06E2D89DEA99A2196CC16DD068CF728
:1003300080E060E081DE89CF1A2DA3CFDA2C1B2D5F
:10034000BA1408F09ECFF8CF0D2DDB2CAB1408F0BB
:1003500094CFF4CF982E0C2DCD1408F08ACFF4CF83
:100360004F5F5F4FB7CFEF92FF920F931F9384B30E
:100370008F6084BBA998AA98AB9AA89AA89880ED98
:1003800097E00197F1F7A89AAB9AAA9AAB9A80E006
:1003900061E052DE80E061E14FDE80E063E04CDE50
:1003A00080E29EE40197F1F780E069E245DE80E0BB
:1003B00063E142DE80E065E23FDE81E06DE23CDE4B
:1003C00080E06AE239DE81E060E036DE81E063E809
:1003D00033DE80E06BE230DE81E060E02DDE81E044
:1003E00063E82ADE80E06AE327DE81E063E024DE62
:1003F00000E117E2C8010197F1F780E06CE21CDE32
:10040000C8010197F1F780E068E216DE80E060E065
:1004100043E823E801E0EE24FF24F4DE80E069E213
:100420000BDE1F910F91FF90EF9008954F925F9216
:100430007F928F929F92AF92BF92CF92DF92EF9274
:10044000FF920F931F93CF93DF93782EA62EF42E57
:10045000E901642F6A0DA90123DE6A2D6F19872D2A
:10046000AE011EDE8F2D870D6A2DAE0119DE872DA0
:100470008F196A2DAE0114DEFF2009F456C08F2DAE
:1004800090E021E0C22ED12CC81AD90A880F991FFA
:1004900044245524481A590ABF2CEE2413E0812E17
:1004A000912C06C0C80CD91C82E090E0880E991EE1
:1004B000D7FC07C0BA9482E090E0480E591EC40CE5
:1004C000D51CE394FE2CF70C1B2D1A0D8F2D612FDC
:1004D000AE01E6DD072D0E19802F612FAE01E0DDA4
:1004E0001A2D1B198F2D612FAE01DADD802F612FA0
:1004F000AE01D6DDFB2CF70C1E2D1A0D8F2D612FB2
:10050000AE01CEDD072D0B19802F612FAE01C8DDA6
:100510001A2D1E198F2D612FAE01C2DD802F612F84
:10052000AE01BEDDEB1408F4BDCFDF91CF911F917A
:100530000F91FF90EF90DF90CF90BF90AF909F9082
:100540008F907F905F904F900895EF92FF920F935E
:100550001F93CF93DF9307DF20E137E2C8ECD0E0B1
:100560002115310509F08FC084E162E344E124E6FE
:1005700000EF1FE0B8DD85E162E345E124E6B3DD8D
:1005800086E162E346E124E6AEDD87E162E347E12E
:1005900024E6A9DD8EE162E34EE124E60FE010E0FF
:1005A000A2DD8FE162E34FE124E69DDD80E262E3BC
:1005B00040E224E698DD81E262E341E224E693DD55
:1005C00082E262E342E224E68EDD83E262E343E21A
:1005D00024E689DD20E43CE9CE010197F1F72150C2
:1005E0003040D1F784E164E148E228E201E0F0EF35
:1005F000EF2EF12C07DE20E533ECCE010197F1F769
:1006000021503040D1F788E268E24CE32CE300E06F
:10061000E12CEFE0FE2EF6DD20E533ECCE01019774
:10062000F1F721503040D1F78CE36CE340E520E551
:1006300001E07AE6E72E7FE0F72EE4DD20E533ECFB
:10064000CE010197F1F721503040D1F780E568E203
:1006500043E824E601E05FEFE52E5FE0F52ED2DD12
:1006600020E533ECCE010197F1F721503040D1F76E
:1006700080E060E043E823E801E03FE0E32EF12C76
:10068000C1DD20E137E2CE010197F1F72150304082
:0606900067CFF894FFCFD4
:00000001FF
